Stack Allocation = 8096 bytes

 Ctl3dV2

 Start     Length     Name                   Class
 0001:0000 00021H     WEP_TEXT               CODE
 0002:0000 045B0H     _TEXT                  CODE
 0003:0000 00F18H     INIT_TEXT              CODE
 0004:0000 00010H     NULL                   BEGDATA
 0004:0010 00066H     _DATA                  DATA
 0004:0076 0000EH     CDATA                  DATA
 0004:0084 00000H     XIFB                   DATA
 0004:0084 00000H     XIF                    DATA
 0004:0084 00000H     XIFE                   DATA
 0004:0084 00000H     XIB                    DATA
 0004:0084 00000H     XI                     DATA
 0004:0084 00000H     XIE                    DATA
 0004:0084 00000H     XPB                    DATA
 0004:0084 00000H     XP                     DATA
 0004:0084 00000H     XPE                    DATA
 0004:0084 00000H     XCB                    DATA
 0004:0084 00000H     XC                     DATA
 0004:0084 00000H     XCE                    DATA
 0004:0084 00000H     XCFB                   DATA
 0004:0084 00000H     XCFCRT                 DATA
 0004:0084 00000H     XCF                    DATA
 0004:0084 00000H     XCFE                   DATA
 0004:0084 00000H     XIFCB                  DATA
 0004:0084 00000H     XIFU                   DATA
 0004:0084 00000H     XIFL                   DATA
 0004:0084 00000H     XIFM                   DATA
 0004:0084 00000H     XIFCE                  DATA
 0004:0084 00000H     DBDATA                 DATA
 0004:0084 00002H     CONST                  CONST
 0004:0086 00008H     HDR                    MSG
 0004:008E 000D4H     MSG                    MSG
 0004:0162 00002H     PAD                    MSG
 0004:0164 00001H     EPAD                   MSG
 0004:0166 0010EH     _BSS                   BSS
 0004:0274 00000H     XOB                    BSS
 0004:0274 00000H     XO                     BSS
 0004:0274 00000H     XOE                    BSS
 0004:0274 00000H     XOFB                   BSS
 0004:0274 00000H     XOF                    BSS
 0004:0274 00000H     XOFE                   BSS
 0004:0280 002B2H     c_common               BSS

 Origin   Group
 0004:0   DGROUP

 Address   Export                  Alias

 0002:2D40 BtnWndProc3d            BtnWndProc3d
 0002:02DC CALLWNDPROCFILTERPROC   CALLWNDPROCFILTERPROC
 0002:3A0E ComboWndProc3d          ComboWndProc3d
 0003:01C0 Ctl3dAutoSubclass       Ctl3dAutoSubclass
 0002:08FC Ctl3dAutoSubclassEx     Ctl3dAutoSubclassEx
 0003:0254 Ctl3dColorChange        Ctl3dColorChange
 0002:1106 Ctl3dCtlColor           Ctl3dCtlColor
 0002:1208 Ctl3dCtlColorEx         Ctl3dCtlColorEx
 0002:1234 Ctl3dDlgFramePaint      Ctl3dDlgFramePaint
 0002:1576 Ctl3dDlgProc            Ctl3dDlgProc
 0003:0234 Ctl3dEnabled            Ctl3dEnabled
 0003:0214 Ctl3dGetVer             Ctl3dGetVer
 0002:1980 CTL3DHOOK               CTL3DHOOK
 0002:0A74 Ctl3dIsAutoSubclass     Ctl3dIsAutoSubclass
 0003:0074 Ctl3dRegister           Ctl3dRegister
 0003:01EE Ctl3dSetStyle           Ctl3dSetStyle
 0002:0BAC Ctl3dSubclassCtl        Ctl3dSubclassCtl
 0002:0DBE Ctl3dSubclassCtlEx      Ctl3dSubclassCtlEx
 0002:0E8E Ctl3dSubclassDlg        Ctl3dSubclassDlg
 0002:107E Ctl3dSubclassDlgEx      Ctl3dSubclassDlgEx
 0002:0AD2 Ctl3dUnAutoSubclass     Ctl3dUnAutoSubclass
 0003:00BE Ctl3dUnregister         Ctl3dUnregister
 0002:0BF0 Ctl3dUnsubclassCtl      Ctl3dUnsubclassCtl
 0003:02BA Ctl3dWinIniChange       Ctl3dWinIniChange
 0002:3748 EditWndProc3d           EditWndProc3d
 0002:39D2 ListWndProc3d           ListWndProc3d
 0002:3E84 StaticWndProc3d         StaticWndProc3d
 0001:0000 WEP                     WEP
 0002:459C ___ExportedStub         ___ExportedStub

  Address         Publics by Name

 0000:0000  Imp  ANSINEXT             (USER.472)
 0000:0000  Imp  BEGINPAINT           (USER.39)
 0000:0000  Imp  BITBLT               (GDI.34)
 0002:2D40       BtnWndProc3d
 0000:0000  Imp  CALLNEXTHOOKEX       (USER.293)
 0000:0000  Imp  CALLWINDOWPROC       (USER.122)
 0002:02DC       CALLWNDPROCFILTERPROC
 0000:0000  Imp  CLIENTTOSCREEN       (USER.28)
 0002:3A0E       ComboWndProc3d
 0000:0000  Imp  CREATECOMPATIBLEDC   (GDI.52)
 0000:0000  Imp  CREATEDIBITMAP       (GDI.442)
 0000:0000  Imp  CREATESOLIDBRUSH     (GDI.66)
 0003:01C0       Ctl3dAutoSubclass
 0002:08FC       Ctl3dAutoSubclassEx
 0002:0FD4       CTL3DCHECKSUBCLASSDLG
 0003:0254       Ctl3dColorChange
 0002:1106       Ctl3dCtlColor
 0002:1208       Ctl3dCtlColorEx
 0002:1234       Ctl3dDlgFramePaint
 0002:1576       Ctl3dDlgProc
 0003:0234       Ctl3dEnabled
 0003:0214       Ctl3dGetVer
 0002:1980       CTL3DHOOK
 0002:0A74       Ctl3dIsAutoSubclass
 0003:0074       Ctl3dRegister
 0003:01EE       Ctl3dSetStyle
 0002:0BAC       Ctl3dSubclassCtl
 0002:0DBE       Ctl3dSubclassCtlEx
 0002:0E8E       Ctl3dSubclassDlg
 0002:107E       Ctl3dSubclassDlgEx
 0002:0AD2       Ctl3dUnAutoSubclass
 0003:00BE       Ctl3dUnregister
 0002:0BF0       Ctl3dUnsubclassCtl
 0003:02BA       Ctl3dWinIniChange
 0000:0000  Imp  DEFDLGPROC           (USER.308)
 0000:0000  Imp  DEFWINDOWPROC        (USER.107)
 0000:0000  Imp  DELETEDC             (GDI.68)
 0000:0000  Imp  DELETEOBJECT         (GDI.69)
 0000:0000  Imp  DOS3CALL             (KERNEL.102)
 0000:0000  Imp  DRAWFOCUSRECT        (USER.466)
 0000:0000  Imp  DRAWTEXT             (USER.85)
 0002:3748       EditWndProc3d
 0000:0000  Imp  ENDPAINT             (USER.40)
 0000:0000  Imp  EXCLUDEUPDATERGN     (USER.238)
 0000:0000  Imp  EXTTEXTOUT           (GDI.351)
 0000:0000  Imp  FATALAPPEXIT         (KERNEL.137)
 0000:0000  Imp  FATALEXIT            (KERNEL.1)
 0000:0000  Imp  FINDRESOURCE         (KERNEL.60)
 0000:0000  Imp  FREELIBRARY          (KERNEL.96)
 0000:0000  Imp  FREEPROCINSTANCE     (KERNEL.52)
 0000:0000  Imp  FREERESOURCE         (KERNEL.63)
 0000:0000  Imp  GETCLASSINFO         (USER.404)
 0000:0000  Imp  GETCLASSNAME         (USER.58)
 0000:0000  Imp  GETCLIENTRECT        (USER.33)
 0000:0000  Imp  GETCURRENTTASK       (KERNEL.36)
 0000:0000  Imp  GETDC                (USER.66)
 0000:0000  Imp  GETDEVICECAPS        (GDI.80)
 0000:0000  Imp  GETDOSENVIRONMENT    (KERNEL.131)
 0000:0000  Imp  GETFOCUS             (USER.23)
 0000:0000  Imp  GETMODULEHANDLE      (KERNEL.47)
 0000:0000  Imp  GETMODULEUSAGE       (KERNEL.48)
 0000:0000  Imp  GETPARENT            (USER.46)
 0000:0000  Imp  GETPROCADDRESS       (KERNEL.50)
 0000:0000  Imp  GETPROFILESTRING     (KERNEL.58)
 0000:0000  Imp  GETPROP              (USER.25)
 0000:0000  Imp  GETSYSCOLOR          (USER.180)
 0000:0000  Imp  GETSYSTEMMETRICS     (USER.179)
 0000:0000  Imp  GETTEXTEXTENT        (GDI.91)
 0000:0000  Imp  GETVERSION           (KERNEL.3)
 0000:0000  Imp  GETWINDOW            (USER.262)
 0000:0000  Imp  GETWINDOWDC          (USER.67)
 0000:0000  Imp  GETWINDOWLONG        (USER.135)
 0000:0000  Imp  GETWINDOWRECT        (USER.32)
 0000:0000  Imp  GETWINDOWTEXT        (USER.36)
 0000:0000  Imp  GETWINDOWTEXTLENGTH  (USER.38)
 0000:0000  Imp  GETWINDOWWORD        (USER.133)
 0000:0000  Imp  GETWINFLAGS          (KERNEL.132)
 0000:0000  Imp  GLOBALADDATOM        (USER.268)
 0000:0000  Imp  GLOBALDELETEATOM     (USER.269)
 0000:0000  Imp  GLOBALREALLOC        (KERNEL.16)
 0000:0000  Imp  GLOBALSIZE           (KERNEL.20)
 0000:0000  Imp  GLOBALUNLOCK         (KERNEL.19)
 0000:0000  Imp  HIDECARET            (USER.166)
 0000:0000  Imp  INFLATERECT          (USER.78)
 0000:0000  Imp  INITTASK             (KERNEL.91)
 0000:0000  Imp  INTERSECTCLIPRECT    (GDI.22)
 0000:0000  Imp  INTERSECTRECT        (USER.79)
 0000:0000  Imp  INVALIDATERECT       (USER.125)
 0000:0000  Imp  ISDBCSLEADBYTE       (KERNEL.207)
 0000:0000  Imp  ISICONIC             (USER.31)
 0000:0000  Imp  ISWINDOWENABLED      (USER.35)
 0003:0EE6       LibEntry
 0003:0A30       LIBMAIN
 0002:39D2       ListWndProc3d
 0000:0000  Imp  LOADLIBRARY          (KERNEL.95)
 0000:0000  Imp  LOADRESOURCE         (KERNEL.61)
 0003:0B8C       LOADUIBITMAP
 0000:0000  Imp  LOCALALLOC           (KERNEL.5)
 0000:0000  Imp  LOCALFREE            (KERNEL.7)
 0000:0000  Imp  LocalInit            (KERNEL.4)
 0000:0000  Imp  LOCALREALLOC         (KERNEL.6)
 0000:0000  Imp  LOCALSIZE            (KERNEL.10)
 0000:0000  Imp  LOCKRESOURCE         (KERNEL.62)
 0000:0000  Imp  LOCKSEGMENT          (KERNEL.23)
 0000:0000  Imp  LSTRCMP              (USER.430)
 0000:0000  Imp  LSTRCMPI             (USER.471)
 0000:0000  Imp  OFFSETRECT           (USER.77)
 0000:0000  Imp  PATBLT               (GDI.29)
 0000:0000  Imp  RELEASEDC            (USER.68)
 0000:0000  Imp  REMOVEPROP           (USER.24)
 0004:0004       rsrvptrs
 0000:0000  Imp  SCREENTOCLIENT       (USER.29)
 0000:0000  Imp  SELECTOBJECT         (GDI.45)
 0000:0000  Imp  SENDMESSAGE          (USER.111)
 0000:0000  Imp  SETBKCOLOR           (GDI.1)
 0000:0000  Imp  SETBKMODE            (GDI.2)
 0000:0000  Imp  SETPROP              (USER.26)
 0000:0000  Imp  SETTEXTCOLOR         (GDI.9)
 0000:0000  Imp  SETWINDOWLONG        (USER.136)
 0000:0000  Imp  SETWINDOWSHOOKEX     (USER.291)
 0000:0000  Imp  SHOWCARET            (USER.167)
 0002:3E84       StaticWndProc3d
 0000:0000  Imp  UNHOOKWINDOWSHOOKEX  (USER.292)
 0000:0000  Imp  UNLOCKSEGMENT        (KERNEL.24)
 0000:0000  Imp  VALIDATERECT         (USER.127)
 0001:0000       WEP
 0004:0029       _aseghi
 0004:0027       _aseglo
 0004:0166       _edata
 0004:0532       _end
 0004:003E       _errno
 0004:0280       _g3d
 0002:30F6       _ListEditPaint3d
 0002:0010       _mpctcdef
 0002:00B8       _mpicvSysColor
 0002:3784       _SharedListWndProc
 0002:3580       _ShareEditComboWndProc3d
 0002:3BFC       _StaticPaint
 0002:3A7C       _StaticPrint
 0004:001A       _STKHQQ
 0000:9876  Abs  __acrtmsg
 0000:9876  Abs  __acrtused
 0000:D6D6  Abs  __aDBdoswp
 0004:0070       __adbgmsg
 0000:D6D6  Abs  __aDBused
 0002:40E8       __aFlshl
 0002:40F4       __aFulshr
 0000:0000  Imp  __AHINCR             (KERNEL.114)
 0004:0030       __aintdiv
 0004:0072       __amblksiz
 0002:4358       __amsg_exit
 0002:4100       __aNlshl
 0002:410C       __aNulshr
 0002:4044       __astart
 0002:41C8       __cexit
 0004:006D       __child
 0002:4192       __cinit
 0002:4350       __cintDIV
 0004:0049       __cpumode
 0002:421B       __ctermsub
 0002:41D2       __c_exit
 0004:0026       __dllinit
 0004:004A       __doserrno
 0004:0166       __edata
 0004:0532       __end
 0004:0066       __environ
 0004:006F       __exitflag
 0004:0034       __fac
 0002:4266       __FF_MSGBANNER
 0002:448D       __findlast
 0002:4118       __fmemcmp
 0004:0078       __fpinit
 0000:9876  Abs  __fptaskdata
 0002:431C       __fptrap
 0002:44AE       __GetDGROUP
 0002:4398       __growseg
 0004:001C       __hModule
 0002:4427       __incseg
 0004:0022       __lpszCmdLine
 0002:4322       __myalloc
 0002:434E       __nearstub
 0004:004C       __nfile
 0002:4512       __nfree
 0002:44BE       __nmalloc
 0002:42E6       __NMSG_TEXT
 0002:4311       __NMSG_WRITE
 0002:458C       __nmsize
 0002:40CF       __nomain
 0002:4528       __nrealloc
 0004:004A       __oserr
 0004:004E       __osfile
 0004:0045       __osmajor
 0004:0044       __osminor
 0004:0048       __osmode
 0004:0044       __osver
 0004:0046       __osversion
 0004:0068       __pgmptr
 0004:0074       __pnhNearHeap
 0002:427C       __setenvp
 0000:0000  Abs  __sizec
 0000:0000  Abs  __sized
 0002:4174       __stubmain
 0004:0040       __umaskval
 0004:001E       __wDataSeg
 0002:4000       __wflags
 0004:0020       __wHeapSize
 0000:0000  Imp  __WINFLAGS           (KERNEL.178)
 0004:0043       __winmajor
 0004:0042       __winminor
 0004:0042       __winver
 0004:002D       ___aDBrterr
 0004:002B       ___aDBswpflg
 0004:0062       ___argc
 0004:0064       ___argv
 0002:459C       ___ExportedStub

  Address         Publics by Value

 0000:0000  Imp  LocalInit            (KERNEL.4)
 0000:0000  Imp  GETWINDOWLONG        (USER.135)
 0000:0000  Imp  SETWINDOWLONG        (USER.136)
 0000:0000  Imp  FREELIBRARY          (KERNEL.96)
 0000:0000  Imp  SELECTOBJECT         (GDI.45)
 0000:0000  Imp  SHOWCARET            (USER.167)
 0000:0000  Imp  GETTEXTEXTENT        (GDI.91)
 0000:0000  Imp  GETCLASSNAME         (USER.58)
 0000:0000  Imp  LOADRESOURCE         (KERNEL.61)
 0000:0000  Imp  LOCALALLOC           (KERNEL.5)
 0000:0000  Imp  GETPARENT            (USER.46)
 0000:0000  Imp  FATALEXIT            (KERNEL.1)
 0000:0000  Imp  CREATEDIBITMAP       (GDI.442)
 0000:0000  Imp  LOCKRESOURCE         (KERNEL.62)
 0000:0000  Imp  DRAWFOCUSRECT        (USER.466)
 0000:0000  Imp  DOS3CALL             (KERNEL.102)
 0000:0000  Imp  GETMODULEUSAGE       (KERNEL.48)
 0000:0000  Imp  CALLWINDOWPROC       (USER.122)
 0000:0000  Imp  FREEPROCINSTANCE     (KERNEL.52)
 0000:0000  Imp  ISICONIC             (USER.31)
 0000:0000  Imp  FINDRESOURCE         (KERNEL.60)
 0000:0000  Imp  __WINFLAGS           (KERNEL.178)
 0000:0000  Imp  GETWINFLAGS          (KERNEL.132)
 0000:0000  Imp  ENDPAINT             (USER.40)
 0000:0000  Imp  GETPROP              (USER.25)
 0000:0000  Imp  SETPROP              (USER.26)
 0000:0000  Imp  GETMODULEHANDLE      (KERNEL.47)
 0000:0000  Imp  FREERESOURCE         (KERNEL.63)
 0000:0000  Imp  GETCLASSINFO         (USER.404)
 0000:0000  Imp  GETWINDOWDC          (USER.67)
 0000:0000  Imp  SETBKCOLOR           (GDI.1)
 0000:0000  Imp  EXTTEXTOUT           (GDI.351)
 0000:0000  Imp  SETBKMODE            (GDI.2)
 0000:0000  Imp  UNHOOKWINDOWSHOOKEX  (USER.292)
 0000:0000  Imp  ISDBCSLEADBYTE       (KERNEL.207)
 0000:0000  Imp  INTERSECTCLIPRECT    (GDI.22)
 0000:0000  Imp  __AHINCR             (KERNEL.114)
 0000:0000  Imp  GLOBALREALLOC        (KERNEL.16)
 0000:0000  Imp  SENDMESSAGE          (USER.111)
 0000:0000  Imp  BITBLT               (GDI.34)
 0000:0000  Imp  LOCALREALLOC         (KERNEL.6)
 0000:0000  Imp  UNLOCKSEGMENT        (KERNEL.24)
 0000:0000  Imp  DRAWTEXT             (USER.85)
 0000:0000  Imp  VALIDATERECT         (USER.127)
 0000:0000  Imp  REMOVEPROP           (USER.24)
 0000:0000  Imp  PATBLT               (GDI.29)
 0000:0000  Abs  __sized
 0000:0000  Abs  __sizec
 0000:0000  Imp  CLIENTTOSCREEN       (USER.28)
 0000:0000  Imp  CREATESOLIDBRUSH     (GDI.66)
 0000:0000  Imp  GETDEVICECAPS        (GDI.80)
 0000:0000  Imp  LOADLIBRARY          (KERNEL.95)
 0000:0000  Imp  SETTEXTCOLOR         (GDI.9)
 0000:0000  Imp  GETPROFILESTRING     (KERNEL.58)
 0000:0000  Imp  INITTASK             (KERNEL.91)
 0000:0000  Imp  GLOBALUNLOCK         (KERNEL.19)
 0000:0000  Imp  RELEASEDC            (USER.68)
 0000:0000  Imp  DELETEDC             (GDI.68)
 0000:0000  Imp  LOCALSIZE            (KERNEL.10)
 0000:0000  Imp  INVALIDATERECT       (USER.125)
 0000:0000  Imp  GETCLIENTRECT        (USER.33)
 0000:0000  Imp  SETWINDOWSHOOKEX     (USER.291)
 0000:0000  Imp  FATALAPPEXIT         (KERNEL.137)
 0000:0000  Imp  GETWINDOWTEXTLENGTH  (USER.38)
 0000:0000  Imp  LSTRCMP              (USER.430)
 0000:0000  Imp  GETVERSION           (KERNEL.3)
 0000:0000  Imp  LOCKSEGMENT          (KERNEL.23)
 0000:0000  Imp  LOCALFREE            (KERNEL.7)
 0000:0000  Imp  INFLATERECT          (USER.78)
 0000:0000  Imp  GLOBALADDATOM        (USER.268)
 0000:0000  Imp  SCREENTOCLIENT       (USER.29)
 0000:0000  Imp  CALLNEXTHOOKEX       (USER.293)
 0000:0000  Imp  GETWINDOW            (USER.262)
 0000:0000  Imp  GETWINDOWWORD        (USER.133)
 0000:0000  Imp  GETPROCADDRESS       (KERNEL.50)
 0000:0000  Imp  GETDC                (USER.66)
 0000:0000  Imp  GETWINDOWRECT        (USER.32)
 0000:0000  Imp  EXCLUDEUPDATERGN     (USER.238)
 0000:0000  Imp  ANSINEXT             (USER.472)
 0000:0000  Imp  GETDOSENVIRONMENT    (KERNEL.131)
 0000:0000  Imp  GLOBALSIZE           (KERNEL.20)
 0000:0000  Imp  HIDECARET            (USER.166)
 0000:0000  Imp  INTERSECTRECT        (USER.79)
 0000:0000  Imp  ISWINDOWENABLED      (USER.35)
 0000:0000  Imp  BEGINPAINT           (USER.39)
 0000:0000  Imp  OFFSETRECT           (USER.77)
 0000:0000  Imp  LSTRCMPI             (USER.471)
 0000:0000  Imp  DEFWINDOWPROC        (USER.107)
 0000:0000  Imp  DEFDLGPROC           (USER.308)
 0000:0000  Imp  GETWINDOWTEXT        (USER.36)
 0000:0000  Imp  GETSYSTEMMETRICS     (USER.179)
 0000:0000  Imp  GLOBALDELETEATOM     (USER.269)
 0000:0000  Imp  GETFOCUS             (USER.23)
 0000:0000  Imp  CREATECOMPATIBLEDC   (GDI.52)
 0000:0000  Imp  DELETEOBJECT         (GDI.69)
 0000:0000  Imp  GETCURRENTTASK       (KERNEL.36)
 0000:0000  Imp  GETSYSCOLOR          (USER.180)
 0000:9876  Abs  __fptaskdata
 0000:9876  Abs  __acrtused
 0000:9876  Abs  __acrtmsg
 0000:D6D6  Abs  __aDBdoswp
 0000:D6D6  Abs  __aDBused
 0001:0000       WEP
 0002:0010       _mpctcdef
 0002:00B8       _mpicvSysColor
 0002:02DC       CALLWNDPROCFILTERPROC
 0002:08FC       Ctl3dAutoSubclassEx
 0002:0A74       Ctl3dIsAutoSubclass
 0002:0AD2       Ctl3dUnAutoSubclass
 0002:0BAC       Ctl3dSubclassCtl
 0002:0BF0       Ctl3dUnsubclassCtl
 0002:0DBE       Ctl3dSubclassCtlEx
 0002:0E8E       Ctl3dSubclassDlg
 0002:0FD4       CTL3DCHECKSUBCLASSDLG
 0002:107E       Ctl3dSubclassDlgEx
 0002:1106       Ctl3dCtlColor
 0002:1208       Ctl3dCtlColorEx
 0002:1234       Ctl3dDlgFramePaint
 0002:1576       Ctl3dDlgProc
 0002:1980       CTL3DHOOK
 0002:2D40       BtnWndProc3d
 0002:30F6       _ListEditPaint3d
 0002:3580       _ShareEditComboWndProc3d
 0002:3748       EditWndProc3d
 0002:3784       _SharedListWndProc
 0002:39D2       ListWndProc3d
 0002:3A0E       ComboWndProc3d
 0002:3A7C       _StaticPrint
 0002:3BFC       _StaticPaint
 0002:3E84       StaticWndProc3d
 0002:4000       __wflags
 0002:4044       __astart
 0002:40CF       __nomain
 0002:40E8       __aFlshl
 0002:40F4       __aFulshr
 0002:4100       __aNlshl
 0002:410C       __aNulshr
 0002:4118       __fmemcmp
 0002:4174       __stubmain
 0002:4192       __cinit
 0002:41C8       __cexit
 0002:41D2       __c_exit
 0002:421B       __ctermsub
 0002:4266       __FF_MSGBANNER
 0002:427C       __setenvp
 0002:42E6       __NMSG_TEXT
 0002:4311       __NMSG_WRITE
 0002:431C       __fptrap
 0002:4322       __myalloc
 0002:434E       __nearstub
 0002:4350       __cintDIV
 0002:4358       __amsg_exit
 0002:4398       __growseg
 0002:4427       __incseg
 0002:448D       __findlast
 0002:44AE       __GetDGROUP
 0002:44BE       __nmalloc
 0002:4512       __nfree
 0002:4528       __nrealloc
 0002:458C       __nmsize
 0002:459C       ___ExportedStub
 0003:0074       Ctl3dRegister
 0003:00BE       Ctl3dUnregister
 0003:01C0       Ctl3dAutoSubclass
 0003:01EE       Ctl3dSetStyle
 0003:0214       Ctl3dGetVer
 0003:0234       Ctl3dEnabled
 0003:0254       Ctl3dColorChange
 0003:02BA       Ctl3dWinIniChange
 0003:0A30       LIBMAIN
 0003:0B8C       LOADUIBITMAP
 0003:0EE6       LibEntry
 0004:0004       rsrvptrs
 0004:001A       _STKHQQ
 0004:001C       __hModule
 0004:001E       __wDataSeg
 0004:0020       __wHeapSize
 0004:0022       __lpszCmdLine
 0004:0026       __dllinit
 0004:0027       _aseglo
 0004:0029       _aseghi
 0004:002B       ___aDBswpflg
 0004:002D       ___aDBrterr
 0004:0030       __aintdiv
 0004:0034       __fac
 0004:003E       _errno
 0004:0040       __umaskval
 0004:0042       __winver
 0004:0042       __winminor
 0004:0043       __winmajor
 0004:0044       __osver
 0004:0044       __osminor
 0004:0045       __osmajor
 0004:0046       __osversion
 0004:0048       __osmode
 0004:0049       __cpumode
 0004:004A       __doserrno
 0004:004A       __oserr
 0004:004C       __nfile
 0004:004E       __osfile
 0004:0062       ___argc
 0004:0064       ___argv
 0004:0066       __environ
 0004:0068       __pgmptr
 0004:006D       __child
 0004:006F       __exitflag
 0004:0070       __adbgmsg
 0004:0072       __amblksiz
 0004:0074       __pnhNearHeap
 0004:0078       __fpinit
 0004:0166       __edata
 0004:0166       _edata
 0004:0280       _g3d
 0004:0532       __end
 0004:0532       _end

Program entry point at 0003:0ee6
